S01300006B6162656C7465737465722E737265637B
S11300000AC021C020C01FC01EC01DC01CC01BC010
S11300101AC019C018C011241FBE20E0A89521BD24
S113002020E025BFE4E6F3E0A0E6B0E003C0C89515
S113003031960D92A237D9F7A2E7B0E001C01D9224
S1130040A537E9F7C9C000C01895CF93DF93CDB7A2
S1130050DEB725970FB6F894DEBF0FBECDBF1B8267
S113006019821A8289819A8127E2803192070CF0E1
S11300700FC08827839B83958C838C81882311F000
S113008081E08B8389819A81019689839A83EACF5F
S11300908B81882359F01D8280917400882311F488
S11300A081E08D832D81209374001FC080917400A2
S11300B08823B1F08091720090917300019790931E
S11300C07300809372008091720090917300992361
S11300D064F487E090E0909373008093720005C00D
S11300E080917000865F8093700080917000853FDE
S11300F018F084EF80937000829BFECF839BFECF29
S113010025960FB6F894DEBF0FBECDBFDF91CF9119
S11301100895CF93DF93CDB7DEB725970FB6F89444
S1130120DEBF0FBECDBF1B8219821A8289819A81DC
S113013027E2803192070CF00FC08827829B8395B9
S11301408C838C81882311F081E08B8389819A814F
S1130150019689839A83EACF8B81882359F01D8283
S113016080917400882311F481E08D832D81209384
S113017074001EC0809174008823A9F080917200DD
S11301809091730001969093730080937200809114
S11301907200909173008830910554F010927300AE
S11301A01092720005C0809170008A508093700094
S11301B0809170008A3018F48AE080937000829BEA
S11301C0FECF839BFECF25960FB6F894DEBF0FBEFD
S11301D0CDBFDF91CF910895CDEDD0E0DEBFCDBF8F
S11301E08FE187BB83E781BB18BA8CE082BB109296
S11301F0730010927200109274008091740088232E
S1130200A1F4809172009091730001969093730011
S113021080937200809172009091730088309105F0
S113022024F01092730010927200809172009091E9
S11302307300805A9F4FF92FE82F8081886187BB14
S1130240809172009091730088599F4FF92FE82F85
S1130250808181BB1982998180917000981708F080
S1130260CCCF8091720090917300805A9F4FF92FE8
S1130270E82F808188BB8091720090917300885927
S11302809F4FF92FE82F80818C6082BB1AD088277A
S1130290829B83958A838A81882309F0D6DE882706
S11302A0839B83958A838A81882309F032DF80E1E6
S11302B088BB8CE082BB05D089818F5F8983CBCFDB
S11302C0FFCFCF93DF93CDB7DEB722970FB6F89465
S11302D0DEBF0FBECDBF19821A8289819A8123E0C5
S11302E0883E92070CF006C089819A810196898321
S11302F09A83F3CF22960FB6F894DEBF0FBECDBF1C
S1130300DF91CF910895CF93DF93CDB7DEB72497D4
S11303100FB6F894DEBF0FBECDBF1B821C828B814B
S11303209C818F3091050CF014C019821A82898146
S11303309A8127E28031920734F08B819C81019667
S11303408B839C83ECCF89819A81019689839A83DC
S1130350EECF24960FB6F894DEBF0FBECDBFDF916B
S1070360CF91089598
S1130364000000000001020401021020400000000B
S105037464001F
S9030000FC
